:0520E20032393143001A
:101FD700AF8475840F75E10343E20443E3C075A43E
:101FE7000F7580F075A51775AD17E4F5A675A7F001
:021FF7008F84D5
:011FF90022C5
:10208300AF84E4F584759D0443F808759A40D2F84B
:022093008F8438
:012095002228
:0620D700122056022083D6
:0520DD00121FD7D32201
:101EF700C200C201C20275FFDE75FFAD1220DD927E
:101F07000030005A1220D77BFF7A2079E21219EEAF
:101F1700EF24FF92013001127D007C14E4FFFE12D2
:101F27001FB0E4FFFE121B2C80217BFF7A2079E291
:101F3700121C67EF24FF92023002107D007C14E42C
:101F4700FFFE121FB0E4FFFE12181AE4FFFE0FBFD8
:101F570000010EBE27F8BF10F5E4F584F5C080FE3A
:102096002321323030454655002324323030454620
:0220A6005500E3
:10205600AF8475840F758A83E4F597F58475C0445B
:0720660075CFE4C2C38F84B3
:01206D002250
:06201C008F27AD27AF265F
:022022008D3DF2
:10202400121FFAEFC454F0F53EAF3D121FFAEF252C
:042034003EF53EFF38
:012038002285
:101FB0008F828E83D3E5829DE5839C501943B701C0
:101FC000758F03E4F0F58F53B7FE2582F582740414
:061FD0003583F58380DE7D
:011FD60022E8
:021D8800A907A9
:101D8A0020C3FD20C5FAC2C4D2C5E4FFFC30C3FD9E
:101D9A0030C3FDE5C154F8FA64086003BA1011E5CE
:101DAA0045BF01044401800254FEF5C27C01807CD7
:101DBA00BA180B8544C27C02C2C4C2C5806EBA205E
:101DCA00028038EA64287030B9010CBC020280151E
:101DDA00EC6404701F8019BC02088BC27C03C2C564
:101DEA008012BC03088DC27C04C2C58007BC0404EF
:101DFA00D2C57F01C2C48034BA300AD2C4D2C57CEB
:101E0A0009E4FF8027BA3802801EBA4006C2C2C25D
:101E1A00C58019BA48028010BA50028003BA58081D
:101E2A00D2C47C08AEC28004D2C4D2C5C2C3EC6498
:081E3A00086003021D9AAF06C7
:011E4200227D
:1020B900AE05AD078E448B45E4FB7F01121D8822D6
:1020A800AE03AB05AD078E447545A07F02121D88AF
:0120B8002205
:0619EE008B218A228923EF
:1019F400752BFF752C20752D96752801752900759A
:101A04002A00E4F527F526F525F524E47F50FEFDAC
:101A1400FCAB27AA26A925A824C3121E9B5036AFC7
:101A2400277BA0E4FD1220B9AB28052AE52AAA29C0
:101A34007002052914F9EF121E89E4FAF9F8E52772
:101A44002401F527EA3526F526E93525F525E83577
:101A540024F52480B6AB2BAA2CA92D121E43FF908B
:101A64000000E06F7062900001121E5CFF900001A4
:101A7400E06F7054900002121E5CFF900002E06F51
:101A84007046900003121E5CFF900003E06F7038F4
:101A9400900004121E5CFF900004E06F702A900016
:101AA40005121E5CFF900005E0B5071C90000612AD
:101AB4001E5CFF900006E0B5070E900007121E5C46
:101AC400FF900007E06F60037F0022AB21AA22A9E8
:101AD40023121E43FF900011E06F702A9000011240
:101AE4001E5CFF900012E0B5071C900002121E5C01
:101AF400FF900013E0B5070E900003121E5CFF90E8
:101B04000014E06F60037F0022900009E0F50CA34D
:101B1400E0F50EA3E0F50F900019E0F508A3E0F559
:071B24000AA3E0F50B7F01AD
:011B2B002297
:0D2039008F26AF31AE3012206E8E308F3109
:02204600AC06E6
:0D204800AB07AF04AD07AF03AB091220B921
:012055002268
:0E20C900E50DC3950C500605090509050D220D
:10206E000FBF00010ED3EF950FEE950E4006122016
:05207E00C9E4FEFF2291
:041B2C008E218F2255
:101B3000E4F526F527F52CF52DF52EF52FF530F5E6
:101B400031850A30850B31850809F527F526750D95
:101B500001E4F52BE526643A6016AF31AE30122071
:101B6000468F26AF31AE3012206E8E308F3180E43A
:101B7000052DE52D7002052CAF31AE301220461236
:101B800020398F27AD27AF261220228F2985292BB8
:101B900012203B1220398F27AD27AF261220227545
:101BA0002E008F2FEF252BF52BE52F752F00F52E0F
:101BB00012203B1220398F27AD27AF26122022EFAB
:101BC000422F852E23852F24E52F252BF52B122040
:101BD0003B1220398F27AD27AF261220228F28E510
:101BE00028252BF52BE528705CF525E525C39529DF
:101BF000505312203B1220398F27AD27AF261220D9
:101C0000228F2AE52A252BF52BC3E5249522E523EF
:101C10009521402DAE23AF24BEFB06BFFE0343B18A
:101C20003043B701758F01852482852383E52AF02F
:101C3000E4F58F53B7FE75B1110524E52470020554
:101C400023052580A612203B1220398F27AD27AF10
:101C5000261220228F2AE52A252B700AE528640106
:061C60006003021B51228B
:011C6600225B
:061C67008B218A22892373
:101C6D00752BFF752C20752D9F7528017529007515
:101C7D002A50E4F527F526F525F524E47F2BFEFD06
:101C8D00FCAB27AA26A925A824C3121E9B5035AF4D
:101C9D0027E4FBFD1220A8AB28052AE52AAA297006
:101CAD0002052914F9EF121E89E4FAF9F8E5272443
:101CBD0001F527EA3526F526E93525F525E83524FC
:101CCD00F52480B7AB2BAA2CA92D121E43FF900033
:101CDD0050E06F7062900001121E5CFF900051E0A9
:101CED006F7054900002121E5CFF900052E06F70F6
:101CFD0046900003121E5CFF900053E06F70389009
:101D0D000004121E5CFF900054E06F702A900005D5
:101D1D00121E5CFF900055E0B5071C900006121EC8
:101D2D005CFF900056E0B5070E900007121E5CFF99
:101D3D00900057E06F60037F0022AB21AA22A923F8
:101D4D00121E43FF90005FE06F702A900001121E7B
:101D5D005CFF900060E0B5071C900002121E5CFF56
:101D6D00900061E0B5070E900003121E5CFF90001D
:0A1D7D0062E06F60037F00227F0127
:011D87002239
:101F6700E48F34F533F532F531AE33AD32AC317839
:101F770008121EC48F348E338D328C317835121E81
:011F8700D782
:081F88008F408E3F8D3E8C3D21
:101F9000AA077808121EB1A907AF40AE3FAD3EAC0C
:0F1FA0003D7810121EB1AB07AF02AD011220A8A1
:011FAF00220F
:04181A008E218F226A
:10181E00E4F526F527F534F533F532F531F538F5DF
:10182E0037F536F535F53CF53BF53AF53975382B88
:10183E00F537F536F535F527F526F52CE4F52BE5D8
:10184E0026643A6007121F838F2680F3E53C24013D
:10185E00F53CE4353BF53BE4353AF53AE43539F5FC
:10186E0039121F838F26121F8312201C8F29852960
:10187E002B121F838F26121F8312201CE48F30F52C
:10188E002FF52EF52DEF252BF52BAE2FAD2EAC2DE6
:10189E007808121EC48F308E2F8D2E8C2D121F8322
:1018AE008F26121F8312201CE5304FF530E52FF5E1
:1018BE002FE52EF52EE52DF52D852F23853024E5EC
:1018CE0030252BF52B121F838F26121F8312201CFF
:1018DE008F28E528252BF52BE5286404703B121F75
:1018EE00838F26121F8312201C121F678F26121F32
:1018FE008312201CE5344FF534E533F533E532F52C
:10190E0032E531F531AF34AE33AD32FC7810121E04
:10191E00C48F348E338D328C31E5286402703B12C5
:10192E001F838F26121F8312201C121F678F2612F1
:10193E001F8312201CE5344FF534E533F533E532C1
:10194E00F532E531F531AF34AE33AD32FC780412F9
:10195E001EC48F348E338D328C31E5342524F5241C
:10196E00E5333523F523E5287058F525E525C39590
:10197E0029504F121F838F26121F8312201C8F2A6D
:10198E00E52A252BF52BC3E5249522E52395214049
:10199E002DAE23AF24BEFB06BFFE0343B13043B7CB
:1019AE0001758F01852482852383E52AF0E4F58F66
:1019BE0053B7FE75B1110524E524700205230525E4
:1019CE0080AA121F838F26121F8312201C8F2AE5D6
:0F19DE002A252B700AE5286401600302184A22AB
:0119ED0022D7
:03000000021800E3
:03000300021A03DB
:03000B00021A06D0
:03001300021A09C5
:03001B00021A0CBA
:03002300021A0FAF
:03002B00021A12A4
:03003300021A1599
:03003B00021A188E
:03004300021A1B83
:03004B00021A1E78
:03005300021A216D
:03005B00021A2462
:03006300021A2757
:03006B00021A2A4C
:03007300021A2D41
:03007B00021A3036
:03008300021A332B
:03008B00021A3620
:03009300021A3915
:03009B00021A3C0A
:0300A300021A3FFF
:10180000787FE4F6D8FD9000007F007E20E4F0A30E
:0A181000DFFCDEFA758145021EF7C9
:101E4300BB010689828A83E0225002E722BBFE029D
:091E5300E32289828A83E49322D0
:101E5C00BB010CE58229F582E5833AF583E022503B
:101E6C0006E92582F8E622BBFE06E92582F8E22285
:0D1E7C00E58229F582E5833AF583E493229F
:101E8900BB010689828A83F0225002F722BBFE0138
:021E9900F32232
:101E9B00EB9FF5F0EA9E42F0E99D42F0EC6480C8BE
:061EAB0064809845F0225E
:101EB100E8600FECC313FCED13FDEE13FEEF13FF0F
:031EC100D8F12233
:101EC400E8600FEFC333FFEE33FEED33FDEC33FC7C
:031ED400D8F12220
:101ED7007401FF3395E0FEFDFC080808E6CF2FF6F6
:101EE70018E6CE3EF618E6CD3DF618E6CC3CF622CF
:101FFA00EF7E0024D0B40A00401624F9B40A004047
:10200A000CB41000400A24E0B41000400374FFFE30
:02201A00FF22A3
:00000001FF
